:18000000000000000000000000000000000000000000000000000000E8
:1000180000000000000000000000000000000000D8
:110040000000000000000000000000000000000000AF
:0100590000A6
:1800630000000000000000000000000000000000000000000000000085
:18007B000000000000000000000000000000000000000000000000006D
:1800930000000000000000000000000000000000000000000000000055
:0300AF000000004E
:0300B60000000047
:18FFE80099B4F0CBF0CAF0CCF080F07FF039F038F037F02DF02CC00033
:18A0000070105010301070301010705030305050707070707070707028
:18A0180070007000500030007020100070403020504070607060706030
:18A03000080808080A0A0A0A0A0A0A0A0A0A0A0A0A0C0C0C0C0C0C0C22
:18A048000C0C0C0C0C0C0E0E0E0E0E0E0E0E0E0E0E0E0E0E0E0E0E10BA
:18A0600010101010101010101010101010101010101010101010101068
:18A07800101010101010101010100E0E0E0E0E0E0E0E0E0E0E0E0E0E6C
:18A090000E0E0E0C0C0C0C0C0C0C0C0C0C0C0C0C0A0A0A0A0A0A0A0AA2
:18A0A8000A0A0A0A0A08080808080808080808080808080806060606DE
:18A0C00006060606060606060606060404040404040404040404040412
:18A0D80004040202020202020202020202020202020200000000000048
:18A0F00000000000000000020202020202020202020202020202020434
:18A10800040404040404040404040404040406060606060606060606CB
:18A1200006060606060808080808080808080808000010001000100081
:18A138007040704070407040704030203020302030203020302030206F
:18A1500030203020302030203020302030203020302030207040704077
:18A16800704070407040100010001000100070207020702070207020BF
:18A1800030003000300030005000500050005000500050005000500087
:18A198005000500050003000300030003000702070207020702070202F
:18A1B000100010001000100070407040704070407040302030203020F7
:18A1C800302030203020302030203020302030203020302030203020BF
:18A1E000302030207040704070407040704010001000100010101010E7
:18A1F800101010101010101010101010101010101010101010101010CF
:18A21000703070307030703070307030703070307030703070307030B6
:18A22800703070307030301030103010301030103010301030103010FE
:18A2400030103010301030103010301030105010501050105010501066
:18A258005010501050105010501050105010501050105010501050106E
:18A27000501050107010701070107010701050105010501050105010B6
:18A288005010501050105010501050105010501050105010501050103E
:18A2A00050105010301030103010301030103010301030103010301066
:18A2B8003010301030103010301030107030703070307030703070304E
:18A2D00070307030703070307030703070307030703010101010101076
:18A2E800101010101010101010101010101010101010101010101010DE
:18A30000101070507050705070507050705070507050705070507050E5
:18A31800705070503030303030303030303030303030303030303030ED
:18A3300030303030303030305050505050505050505050505050505095
:18A348005050505050505050505050505050505050505050505050507D
:18A3600070707070707070707070707070707070707070707070707065
:18A378007070707070707070707070707070707070707070707070704D
:18A39000707050505050505050505050505050505050505050505050F5
:18A3A800505050505050505050505050505050505050303030303030DD
:18A3C000303030303030303030303030303030303030303030307050A5
:18A3D8007050705070507050705070507050705070507050705070506D
:18A3F000101010101010101010101010701070107010701050105010D5
:18A40800501050105010501050105010501050105010501050105010BC
:18A42000501050105010301030103010301030103010301030103010C4
:18A438003010301030103010301030103010301030103010301030100C
:18A4500030103010301030103010301030103010301030103010703094
:18A468007030703070307030703070307030703070307030703070305C
:18A4800070307030703070307030703070307030703070307030703044
:18A498007030703070307030703070307030703070307030703070302C
:18A4B00070307030703070301010101010101010101010101010101014
:18A4C800101010101010101010101010101010101010101010101010FC
:18A4E000101010101010101010101010101010101010101010101010E4
:18A4F800101010101010101010101010101010101010101010101010CC
:18A5100010101010101070507050705070507050705070507050705013
:18A528007050705070507050705070507050705070507050705070501B
:18A5400070507050705070507050705070507050705070507050705003
:18A558007050705070507050705070503030303030303030303030302B
:18A5700030303030303030303030303030303030303030303030303053
:18A588003030303030303030303030303030303030303030303030303B
:18A5A000303030303030303030303030505050505050505050505050A3
:18A5B8005050505050505050505050505050505050505050505050500B
:18A5D000505050505050505050505050505050505050505050505050F3
:18A5E8005050707070707070707070707070707070707070707070701B
:18A60000707070707000700070007000500050005000500050005000E2
:18A618005000500050005000500050005000500050005000500030008A
:18A63000300030003000300030003000300030003000300030003000D2
:18A64800300030003000300030003000300030003000300030003000BA
:18A66000300030003000300030003000300070207020702070207020C2
:18A678007020702070207020702070207020702070207020702070200A
:18A69000702070207020702070207020702070207020702070207020F2
:18A6A800702070207020702070207020702070207020702070207020DA
:18A6C000100010001000100010001000100010001000100010001000C2
:18A6D800100010001000100010001000100010001000100010001000AA
:18A6F00010001000100010001000100010001000100010001000100092
:18A70800100010001000100010001000100010001000100010007040D9
:18A72000704070407040704070407040704070407040704070407040E1
:18A73800704070407040704070407040704070407040704070407040C9
:18A75000704070407040704070407040704070407040704070407040B1
:18A7680070407040302030203020302030203020302030203020302059
:18A7800030203020302030203020302030203020302030203020302001
:18A79800302030203020302030203020302030203020302030203020E9
:18A7B00030203020504050405040504050405040504050405040504051
:18A7C800504050405040504050405040504050405040504050405040B9
:18A7E000504050405040504050405040504050405040706070607060E1
:18A7F8007060706070607060706070607060706070607060201F201FAB
:18A810001E1D1C1B1A191817161514131211102F2E2D2C2B2A29282754
:18A82800262524232221201F1E1D1C1B1A191817161514131211102F7C
:18A840002E2D2C2B2A292827262524232221201F1E1D1C1B1A191817C4
:18A85800161514131211100F0E0D0C0B0A09080738373635343332315C
:18A87000302F2E2D2C2B2A292827262524232221201F1E1D1C1B1A1964
:18A888001817161514131211100F0E0D0C0B0A3534333231302F2E2D00
:18A8A0002C2B2A292827262524232221201F1E1D1C1B1A191817161594
:18A8B80014131211100F302F2E2D2C2B2A292827262524232221201F58
:18A8D0001E1D1C1B1A191817161514131211100F0E0D3231302F2E2DD0
:18A8E8002C2B2A292827262524232221201F1E1D1C1B1A19181716154C
:18A90000142B2A2928272625242322212021201F1E1D1C1B1A19181735
:18A91800161514131211302F2E2D2C2B2A292827262524232221201FEB
:18A930001E1D1C1B1A191817161514131211302F2E2D2C2B2A29282713
:18A94800262524232221201F1E1D1C1B1A191817161514131211100F7B
:18A960000E0D0C0B0A0908393837363534333231302F2E2D2C2B2A2951
:18A978002827262524232221201F1E1D1C1B1A1918171615141312111B
:18A99000100F0E0D0C0B363534333231302F2E2D2C2B2A29282726252B
:18A9A80024232221201F1E1D1C1B1A1918171615141312111031302FE5
:18A9C0002E2D2C2B2A292827262524232221201F1E1D1C1B1A19181743
:18A9D800161514131211100F0E333231302F2E2D2C2B2A292827262531
:18A9F00024232221201F1E1D1C1B1A19181716152C2B2A292827262543
:18AA080024232217808183848687898A8C8D8F909293959698999B9C9E
:18AA20009D9FA0A1A3A4A5A7A8A9AAABACADAFB0B1B2B3B3B4B5B6B711
:18AA3800B8B8B9BABABBBBBCBCBDBDBDBEBEBEBFBFBFBFBFBFBFBFBF53
:18AA5000BFBFBEBEBEBDBDBDBCBCBBBBBABAB9B8B8B7B6B5B4B3B3B286
:18AA6800B1B0AFADACABAAA9A8A7A5A4A3A1A09F9D9C9B999896959391
:18AA800092908F8D8C8A898786848381807E7C7B797876757372706FB7
:18AA98006D6C6A696766646362605F5E5C5B5A58575655545352504FE4
:18AAB0004E4D4C4C4B4A49484747464545444443434242424141414000
:18AAC80040404040404040404040414141424242434344444545464748
:18AAE0004748494A4B4C4C4D4E4F50525354555657585A5B5C5E5F609E
:18AAF8006263646667696A6C6D6F707273757678797B7C7E040505057C
:18AB100005060606070707070808080808080808080707070706060684
:18AB2800050505050404040303030302020202010101010000000101DB
:18AB40000101020202020303030304040404050505060606060707079B
:18AB580007070707070707070707070706060606050505040404040456
:18AB700004030303030202020202020202020202020202020303030393
:18AB88000404040408080A0A0A0C0C0C0E0E0E0E10101010101010109B
:18ABA000100E0E0E0E0C0C0C0A0A0A08080806060604040402020202D5
:14ABB80000000000000000000002020202040404060606085B
:18C000008E1FFFBDE14EBDCED75FBDCE75BDE368BDF022BDF003BDC0CB
:18C0180094CC30D4BDD4A9C601D74A0E72108FBDD6737F006CBDD3CF1B
:18C0300036C603D787CC01FDBDDF12C402968884FD1B9788BDC0C37FC5
:18C04800004AC636BDD7BE3CCE00C8BDD3AA38BDD324BDCD98C601BDAA
:18C06000D4E1867FC610BDE192D688C402BDCE75BDCD7348240A260546
:18C07800BDCD982003BDCDDDBDCE203F4FBDD4E1BDD651BDCD6BBDD3F0
:18C090003A7EC0697F0048C601D74ACECEF9DF4BCE1EF8CCCEF9ED06DF
:18C0A800ED044FED02A701DF44CE0000DF7DDF7FCEFFFFDF81DF8372FE
:18C0C000108F39CEC0C9DF4B39BDD68D4D27037EC12BD69017C4C0C113
:18C0D8008026037EC12B3CCEC161BDE6E938BDD7A35FBDD7803CCE0099
:18C0F000FABDD3AA383CCEC166BDE6E938BDD7A35FBDD7803CCE019092
:18C10800BDD3AA383CCEC15ABDE6E938BDD7A35FBDD78096908A808466
:18C12000BF97903CCE00FABDD3AA38BDC17D3CCE0064BDD3AA38CE0002
:18C138006DBDD627BDD638BDC19EBDE480BDD80A3FDE668C04B025EF4A
:18C15000D6902AEBC47FD79020E5444731594645004D433730003133B2
:18C168002030303100524F4D20494E49540020534C4F545300860097FA
:18C180008B717F937F00897F008A7F00B07F00AF7F009272108FC60241
:18C198008601BDD87639BDE3A94D2A037EC1D937D68B58CEC1BC3A3341
:18C1B0008CC1D62404EE006E007EC1D9C2BDC8ABC720C6F0C7BBC3D90B
:18C1C800C5B8CADCC1E1C1D6C1D6CBE4CCB67EC1D9D6932A14DE8C26EC
:18C1E00010717F93BDD74FC600D78B7F00897F008A3937C6000FD78CF0
:18C1F800C628D78D0E72809333394F4B004E4F204C4F434B20006F755A
:18C2100074206F660052616E6765200077726974696E670073746F72D4
:18C228006564006661696C65640064656C6574696E67005458534849F4
:18C240004654005351204F4E005351204F4646004F4646002573204871
:18C258005A00000B0C0D0E0F10111203060913020508000104070A4D69
:18C27000454E552020202000C68B524543414C4C202000C68B53544FC3
:18C28800524520202000C6F7545820435443535300CBD644544D4620B2
:18C2A00020202000CCA156455253494F4E2000CBBD4445462043482051
:18C2B8002000CA95005896878103270E81022705CEC30C2011CEC3347F
:18C2D000200C96852705CEC2E42003CEC30C3AEE00546E00C652C65295
:18C2E800C652C652C652C652C652C652C652C652C652C35CC375C652F7
:18C30000C652C3C5C1D6C652C652C652C889C889C889C889C889C889C0
:18C31800C889C889C889C889C1D6C35CC375C38EC1D6C3C5C1D6C3D938
:18C33000C684C597C571C56EC543C543C543C543C543C543C597C54352
:18C34800C568C35CC375C38EC1D6C557C63CC3D9C684C1D6DE6F3CDE6F
:18C360006D3CCE0000CC30D4BDDCA730BDD6197EC97D7EC1D9DE6F3CFD
:18C37800DE6D3CCC30D4CE0000BDDCD430BDD6197EC97D7EC1D9D68FFE
:18C390001784202622C410260FC4CFCA10D78F8601C602BDD876201A22
:18C3A800C4CFCA20D78F8602C602BDD876200BC4CFD78F8600C602BD10
:18C3C000D8767EC1D972018FD6952606CC06D6BDEA0CC606D7957EC194
:18C3D800D996932B03BDD73A968B81052752C605D78BBDC1F25FBDD79F
:18C3F000803CCEC23BBDE6E938BDD7A33CCE0064BDD3AA38DE733CDE68
:18C40800713C5FBDD78030A600AA01AA02AA032715BDDD598645C6035F
:18C42000BDE6153838BDD7A3BDD6387EC1D93CCEC250BDE6E93820EBD7
:18C43800BDC1F296878103272181022702201BC1052759C111272FC17D
:18C4500010270CC108261FCE0000DF8C7EC1D97EC4C1C10A273EC1112D
:18C468002714C1132608CE0000DF8C7EC1D937BDD74F337EC2BDBDC166
:18C48000F2DE712612DE73260EDE77DF833CDE75DF813C3F7EC40ACE6B
:18C498000000DF83DF813F3C3C7EC40ACE0071BDDD59DC73DD77DD8392
:18C4B0003736DC71DD75DD8137363F7EC40A7EC1D986125FBDC99D4D93
:18C4C800260220147F008D7F008C7EC1D9D6597C0000CE00B93A6F00F6
:18C4E0003C3C30CC00B9BDD0BDCE00B9BDD10AC103270E4FC105260278
:18C4F800C6045858C3DC872003CCDC9730BDDB73EC00DD75DD81EC0265
:18C51000DD77DD833FC600D78BCC0008DD8C7EC40AD6932B06CE005AAD
:18C52800BDD73ABDC1F25FBDD7805F3C3737866CBDE4B93838BDD7A34E
:18C540007EC1D9CC0320BDECC03CCE0028BDD3AA38BDED0C7EC1D9D62B
:18C5580042CA10D742D716D617C810D7177EC1D9BDEC437EC1D97EC19B
:18C57000D9D6932B06CE005ABDD73ABDC1F25FBDD7804FD68E37363611
:18C5880036866C5FBDE4B93838BDD7A37EC1D9D6932B06CE005ABDD7A5
:18C5A0003ABDC1F25FBDD780C606D78B7F0089CEC26FBDE6E97EC1D98D
:18C5B800BDC1F296878102271B810327022000C1132754C10A276A960B
:18C5D00089C10B2726C10C27187EC1D9C108273FC10527559689C10B31
:18C5E8002711C10C27037EC1D94D27034A260B860620074C8107260253
:18C60000860197895FBDD780CEC26F4D270B08E60026FB0808084A20F9
:18C61800F2BDE6E97EC1D9CEC26F968908E60026FB4D27064A0808086B
:18C6300020F27F0089EE016E007EC1E1D6932B03BDD73A86035FBDC988
:18C648009D4D26037EC9027EC1E1C10A2508C00ACEC67A3AE600969543
:18C66000270BBDEC433CCE0028BDD3AA38BDED25BDEB2BC604D7957EAA
:18C67800C1D90E00000D0C00000A0B0FD6932B1BBDD73A5FBDD7803C99
:18C69000CEC6E7BDE6E9383CCE012CBDD3AA38C602D78BBDC1F2CEC77B
:18C6A800BBDF895FBDD780CE00B9D692BDC833CE84003CCE17D73CCEE9
:18C6C00000B9BDDCEC8604C603BDE615D659C1062409C6208663BDE486
:18C6D800B920F1D6928664BDE4B938387EC1D94D20524543414C4C002C
:18C6F000D6932BAFBDD73A5FBDD7803CCEC717BDE6E9383CCE012CBD0E
:18C70800D3AA38C602D78BCEC7E9DF897EC6AB4D2053544F524520004B
:18C72000BDC1F296878103270481022740C1122773C1132765C10B271B
:18C738004BC10C2754C10A250AC10A27037EC1D97EC1E1375F969281F0
:18C750000A2513C60A8114250DC61430A60081052504337EC1D9321B01
:18C7680097927EC6ABC1082729C112272FC10B270BC10C2714C105276C
:18C78000C77EC1D9D6925CC11925015FD7927EC6ABD6922602C6195A7E
:18C7980020F2DE897F00897F008A6E00D692C10F250AC1142504C01458
:18C7B0002004C60ECB0AD7927EC6ABD692C11924103C3C30BDCEFEBDE8
:18C7C800D619C600D78B7EC97D5FBDD7803CCEC7E0BDE6E9387EC1E176
:18C7E00045727220536C6F74005FBDD780D692C11924DEBDCF584D2747
:18C7F800153CCEC22BBDE6E938BDD7A33CCE01F4BDD3AA3820133CCE74
:18C81000C224BDE6E938BDD7A33CCE0064BDD3AA387EC1E14D454D2030
:18C82800434800534C4F5420257800373C3434860A3DCE01003A183075
:18C840003CCE0002BDDF9C384D262430EC00040404CE04E2BDDABF3764
:18C85800363CCC4780CE19A1BDDCA730EE063233ED003233ED024F31B1
:18C8700031383339373C860A3DCB03CE01003A18CE0006BDDF9C383335
:18C8880039BDD73A4FBDD6DD8601978BBDC1F2CB3017D659CE00B93AB7
:18C8A00016E7008663BDE4B97EC1D9C10A24099659810826DF7EC1D99B
:18C8B800CEC8C3C00A583AEE006E00C8D7C1D6C1D6C1D6C1E1C1D6C1F9
:18C8D000D6C4D5C1D6C8F9BDC1F2BDD720D659CE00B93A6F00860197E8
:18C8E8008B7EC1D9BDC1F24FBDD6DD7F00B97EC1D94FD659C300B91804
:18C900006F003C3C30CC00B9BDD0BDCE00B9BDD10A5D260538387EC1E3
:18C91800E17F008C4F5858C3DC7F30BDDB73CCC999BDDD082506CC00FC
:18C930000ABDD99230BDD619C61ED769CE001586205FBDD3BB16BDD3E4
:18C94800BB5FBDD7807202933F4FBDD6DDD693C40126123CCEC205BDB0
:18C96000E6E9383CCE00C8BDD3AA3820083CCEC202BDE6E9383CCE00B0
:18C97800C8BDD3AA385FBDD780CE006DBDD627BDD7A3BDD638C600D766
:18C990008B717F9338387EC1D91DCD65003716545454543730E601843B
:18C9A8000FA7015D2714C1012708C66137C67A37200EC63037C67A3790
:18C9C0002006C63037C6393730E603378601BDD911BDC1F2BDE480BD0A
:18C9D800D80ABDE3A9DE8C272D4D2BF096878103270AC108277BC105F3
:18C9F000271C2008C1132771C10A2712C10B271AC10C2738C110274AD9
:18CA0800C10D274620C3334FBDD911313131318601393337CE00513A88
:18CA2000A600847F30A10124034C2002A602BDD78016CA808663BDE448
:18CA3800B97EC9D13337CE00513AA600847F4A30A102250220E0A601BE
:18CA500020DC30334FBDD911E10327035A2002E604374CBDD9117EC994
:18CA6800D1334FBDD9113131334FCE00513A3736A600CE00B9333AA7D1
:18CA8000005C086F00173330E10027035C20E3314FCE00B939BDC1F237
:18CA98005FBDD7808607978BD688C402270C3CCECAD1BDE6E938C602DC
:18CAB000200A3CCECACABDE6E938C601D789BDD7A37EC1D953544F5224
:18CAC80045004D414E55414C004155544F00CAC4CACACAD1BDC1F29657
:18CAE000878103270E81022700C1082745C10527152008C113273BC1FE
:18CAF8000A270BC10B270AC10C27267EC1D97EC1E1D6895CC1032601F5
:18CB10005FD7895FBDD780D68958CECAD63AEE00BDE6E9BDD7A37EC18C
:18CB2800D9D6895A2AE3C60220DFD68927325A262B968884FD1B978853
:18CB400016CE01FD3CBDE013384D264B5FBDD780CEC202BDE6E9BDD7F4
:18CB5800A33CCE00C8BDD3AA387EC1E1C60220D1BDCFB84D26295FBD09
:18CB7000D7803CCEC202BDE6E938BDD7A35FBDD7803CCEC224BDE6E99E
:18CB880038BDD7A33CCE03E8BDD3AA387EC1E1364FBDD6DD3CCEC22BB3
:18CBA000BDE6E9383CCE01F4BDD3AA38338678BDE4B93CCE03E8BDD338
:18CBB800AA387EC1E1BDC1F25FBDD7808608978B3CCEC166BDE6E938DB
:18CBD000BDD7A37EC1D9C60BD78BC6FF2006C60AD78BC6FFBDC1F24F2A
:18CBE8005D2B2CC10B270FC10C2716C113276DC10A26667EC1E1D6962A
:18CC0000C13624107C0096200ED6962602C6375AD79620037F00965FC2
:18CC1800BDD780D696C13725015F58CEED823AEC00260D3CCEC250BD40
:18CC3000E6E938BDD7A320293736CE00B9BDE8A132338303E82501082A
:18CC4800E602E703C62EE7025FE704CE00B93CCEC254BDE6E938BDD7DC
:18CC6000A37EC1D9D68BC10B26F7D696272B58CEED823AEC0072048F39
:18CC7800D6852703BDEAB15FBDD7803CCEC202BDE6E938BDD7A33CCE81
:18CC900000C8BDD3AA387EC1E171FB8FBDEC8920DE4FBDD6DD860C971F
:18CCA8008B7EC1D92A303044433030414223C10C271DC10B26037EC175
:18CCC000E1C10A250FC00ACECCAC3AE600C03026037EC1D97EC89472CF
:18CCD800018F9695270DBDEC433CCE0028BDD3AA38200D7D0096270856
:18CCF0003CCE00C8BDD3AA3896595FBDD7801127433736CE00B93AE6F7
:18CD080000C141240EC130240CC12A2704C60F2006C644C006C030BD30
:18CD2000ED25BDEB2BC6208663BDE4B93CCE0064BDD3AA38BDEC433CE5
:18CD3800CE0032BDD3AA3832335C20BA71FE8F7EC1E1D640C802D740C1
:18CD5000D70171FD0339D664C4022702C602964084FD1B974097017106
:18CD6800FD03397D006C260220E4399685D617C48026035F2002C6016F
:18CD8000DA8FC4011126057F0086200BD6865CD786C1142502888139AE
:18CD9800D68FC4042703BDEC89C631BDD7BE86DFC640BDE192C605D774
:18CDB000683FD66826FB86FE5FBDE1925FBDCE980FC602D79471FD938D
:18CDC8000ECE006DBDD53A7F008586FFC680BDE1927F008E39C635BD41
:18CDE000D7BEC601BDCE98CE006DBDD58586FFC601BDE192C605D768E4
:18CDF800D66826FCC62086BFBDE192867F5FBDE192C601D7850FC602DA
:18CE1000D79471FD930ED68FC4042703BDEB1839D68EDA85264EC6053E
:18CE2800D78ED68FC430271196915858D4152720810A27054C979120AA
:18CE400033D643C480262D71F71586FFC680BDE192C635BDD7BE201CF6
:18CE58004D27054A97912014D643C480270E720815867F5FBDE192C628
:18CE700031BDD7BE39961584042601395D2709961594022603BDCFB820
:18CE8800867FC600BDE192866DC600BDE19220FE37363C5D260571DF0F
:18CEA000032003722003383233393C30E3003736EC04EE003C37A80034
:18CEB80016CED1243A3A32E601A800383736083C1830A30438323326B9
:18CED000E33830ED04383937D64237C4EFD742D716D617C41026037EF6
:18CEE800258033D742D716333971FB1739720417393FDE4B6E00373C1D
:18CF0000301883000A1835860A3DCE01003A18303CCE000ABDDF9C3855
:18CF18004D263330EC00040404CE04E2BDDABF37363CCC4780CE19A165
:18CF3000BDDCA730EE0E3233ED003233ED0230EC018401CE61A8BDDAC7
:18CF4800BFDD83DF814F3018C3000A18353833393C37301883000A189D
:18CF600035DE6F3CDE6D3CCC4780CE19A1BDDCD4CC04E2BDD9923832A8
:18CF78003305050530ED00DE733CDE713CCC61A8BDD992383830E702A4
:18CF90008401AA01A7015FE703E60A860A3D3CCE01003A3CCE000A3C16
:18CFA800BDE0863838383018C3000A18353338393C37363C3C37DE6FFB
:18CFC0003CDE6D3CCC4780CE19A1BDDCD4CC04E2BDD99238323305058D
:18CFD8000530ED005F37DC77DE752A0ABDDD363C306C026802383736F6
:18CFF0003CDC71DA73DA74830000270730E604CA04E704CC61A8BDD916
:18D0080092383830E7038401AA00AA02A70231303CCC01FACE0003BD7E
:18D02000E0D64D271038303CCE01FA3CCE00033CBDE0863838383838CD
:18D038003331333839373C3C37303CCC01FACE0003BDDF9C384D2668A3
:18D0500030EC00040404CE04E2BDDABF37363CCE19A1CC4780BDDCA792
:18D0680030EE073233ED003233ED0230EC018401CE61A8BDDABF3736A9
:18D080003C30E605C4022708383233BDDD3620033832333C30EE05EDD3
:18D09800063233ED0430E601EE03C4042609CC0000ED08ED0A2009EC58
:18D0B00006ED0AEC04ED084F33383833393C37364F5FED00ED0238E6D7
:18D0C80000C47F273BC1302504C13A25113C30EE02E600EA01EA02EA5D
:18D0E0000327213820223CC03037CCDC9F30EE03BDDB73334FE302ED49
:18D0F80002CC0000E901E701A900A700380820BF38393C4F5F6D002722
:18D1100006C300010820F638393132333435363738391D0F0000102174
:18D1280020423063408450A560C670E781089129A14AB16BC18CD1ADAF
:18D14000E1CEF1EF123102103273225252B5429472F762D693398318F5
:18D15800B37BA35AD3BDC39CF3FFE3DE246234430420140164E674C737
:18D1700044A45485A56AB54B85289509E5EEF5CFC5ACD58D3653267201
:18D188001611063076D766F6569546B4B75BA77A97198738F7DFE7FE47
:18D1A000D79DC7BC48C458E5688678A70840186128023823C9CCD9ED89
:18D1B800E98EF9AF89489969A90AB92B5AF54AD47AB76A961A710A5053
:18D1D0003A332A12DBFDCBDCFBBFEB9E9B798B58BB3BAB1A6CA67C8715
:18D1E8004CE45CC52C223C030C601C41EDAEFD8FCDECDDCDAD2ABD0B5F
:18D200008D689D497E976EB65ED54EF43E132E321E510E70FF9FEFBEA4
:18D21800DFDDCFFCBF1BAF3A9F598F78918881A9B1CAA1EBD10CC12DA0
:18D23000F14EE16F108000A130C220E3500440257046606783B9939894
:18D24800A3FBB3DAC33DD31CE37FF35E02B1129022F332D242355214B6
:18D2600062777256B5EAA5CB95A88589F56EE54FD52CC50D34E224C354
:18D2780014A004817466644754244405A7DBB7FA879997B8E75FF77EC2
:18D29000C71DD73C26D336F2069116B06657767646155634D94CC96D28
:18D2A800F90EE92F99C889E9B98AA9AB584448657806682718C008E1CE
:18D2C000388228A3CB7DDB5CEB3FFB1E8BF99BD8ABBBBB9A4A755A54F0
:18D2D8006A377A160AF11AD02AB33A92FD2EED0FDD6CCD4DBDAAAD8B56
:18D2F0009DE88DC97C266C075C644C453CA22C831CE00CC1EF1FFF3E44
:18D30800CF5DDF7CAF9BBFBA8FD99FF86E177E364E555E742E933EB265
:18D320000ED11EF0373CD664D765C664D76ACEF057DF46C602D794380F
:18D33800333937363CD665966410273A369B659765D66B270B30A600A7
:18D350005A27034A26FAD76BD669270B30A6005A27034A26FAD769D64A
:18D368008E270B30A6005A27034A26FAD78E33966A102B06976A3832E5
:18D3800033398B64976ADE6608DF66DE8C270309DF8CD69427035AD7DB
:18D3980094D69527E17A009526DCBDEC4371FE8F20D418D363182405F8
:18D3B0009C633F25FB9C633F24FB3936A40011270C32367D00692703DB
:18D3C8003F20F186013239BDD3DB4D2705BDD487860139301883000C78
:18D3E0001835303CCC01FACE0003BDDF9C384D267630EC00040404CE95
:18D3F80004E2BDDABF37363CCC4780CE19A13C30E304ED043233E90388
:18D41000E703A902A702303233ED0C3233ED0E30EC018401CE61A8BDA2
:18D42800DABF373C30E604C40238332711435318435318C3000118C95C
:18D440000089001820003C30ED083233ED0630E601C4042609CC000080
:18D45800ED00ED022009EC06ED02EC04ED004F4D27093018C3000C18FE
:18D4700035201338DF7138DF7338DF7538DF7738DF6D38DF6F4F393C42
:18D488003736CEAF60DF6FCE19D6DF6DCE0000DF71DF73CE0073DF75E6
:18D4A000CEF780DF77323338393C373671F717CEBA003CCE00DB3CBD75
:18D4B800D992323338830000261A3C323384C0261386015FBDE1F332CA
:18D4D00033374F7F00857F008633383932860120F2D615C4204D2619B8
:18D4E800969384022613969426241727028601989384012719860297FA
:18D50000945D260771FE93C6372005720193C633BDD7BE71FD9339D670
:18D5180015C42039DF79DD7B37363CCC007FBDD9921838384FBDE1F395
:18D5300086015FCE0480BDE1F339EC023736EE003CCC89C0CE0146BD75
:18D54800DCD4303CCC30D4BDD9DD3131CC30D404183C30A3003838326D
:18D56000332509C3000118C900890018BDD51CBDD60537363CCE014608
:18D57800CC89C0BDDCA738DF6D38DF6F39EC023736EE003CDC73DE71E0
:18D59000BDDCD4CC30D4BDD992CC30D404183C30A30038383233250920
:18D5A800C3000118D900990018BDD51CBDD60537363CDE71DC73BDDCDF
:18D5C000A738DF6D38DF6F39D68526037ED53A7ED585EC02EE00373637
:18D5D8003CCC30D4BDD992CC30D404183C30A300383832332509C30046
:18D5F0000118D9009900183937363CCC30D4CE0000BDDAFE39DE7B3C9D
:18D60800DE793CCC30D4CE0000BDDAFE31313131393736EC02DD7FECA4
:18D6200000DD7D3F323339EC00EE023C3736866CC603BDE4B938383978
:18D638004FDE71270EDE73270ADE712B04860120028602C606BDD876FF
:18D6500039DE7D270BCE007DBDD5C8CE0000DF7DDE818CFFFF270BDF33
:18D6680071DE83DF73CEFFFFDF8139373686FFC604BDE1923CCE001417
:18D68000BDD3AA3886FB5FBDE192323339BDE37D4D27FACC0000DD6BD3
:18D698004F36BDE37D4D323727F83116C17E271DBDE3D6DC66C30014AA
:18D6B000183CBDE37D384D2604C17E27089C6626F0C6012004BDE3D65B
:18D6C8005F370F7F00B67F00B70E86A8976B8601BDD6DD323937363CF1
:18D6E000C6788670BDE4B97F0059CE0051CC2020ED00ED02ED04ED06E1
:18D6F80030C601E402270B7F004EC67A8670BDE4B930C602E402270C9D
:18D71000C6798670BDE4B9CE0000DF4F3832333937363C4FD6595A37E8
:18D72800BDD780C6208663BDE4B933BDD78038323339DE51DF5ADE53F6
:18D74000DF5CDE55DF5EDE57DF60DE58DF6139CE005A5FBDD780E60082
:18D758003C8663BDE4B93808D659C10825F0E600BDD7803937BDE3E102
:18D77000BDE37D4D26F732333936862A976B323937363C17C47FC1085D
:18D788002415915926057B088F270CD759CB608670BDE4B971F78F381C
:18D7A00032333937363CD65937C6208663BDE4B9D659C10825F333BD9B
:18D7B800D780383233391784338133270C813227048601200686042042
:18D7D00002861036483630964D5D2B20C40C270CC40826126300A4002C
:18D7E800AA01201263006301A400A4012008AA00AA012002A801D64ED0
:18D800001127028A80974D31313937363C4F7C004AD64D584954D74D53
:18D818007A004A4D271C37D84E86035424048D1620075424058D0F203F
:18D8300001544A26EE33C47FD74E3832333937361630A604C103270E66
:18D84800C1022710C633843044444444200CC63184032006C632840CB9
:18D860004444442409CA04442404C4FBCA088670BDE4B93233393C368C
:18D8780037BDDD7B37308103275F8102273D81012711964F16A4002774
:18D890007B6300E400D74FC6002058964F16A4002711965016A40027BC
:18D8A800636300E400D750D64F6300EA00D74FD6506300E400D750C6A5
:18D8C000012030965016A4002709964F16A400263BD650EA00D750D622
:18D8D8004FEA00D74FC6022012964F16A40026A9965016A40026E4D6F1
:18D8F0004F20C0965936378670E601BDD78033CB6D8670BDE4B933CAEC
:18D9080080BDD78031333238393C3637C108241E4D27028680CE00511D
:18D920003AE600C4801B270E3337BDD780E600C8808663BDE4B93332E7
:18D93800383937363C30EE06271A3C30EE02E60037081830ED03EE05AC
:18D9500033E700081830ED04380926E63832333937363CCE00013CCEBF
:18D9680000003C3068076906EC0059492509A3042407E3040C2003A316
:18D98000040DED006903690224E23832333131313139303736EC043756
:18D9980036EC023736CC00003736306F0A6F0B6F0CC601E70D6805697E
:18D9B0000469036902EC0059492509A3062407E3060C2003A3060DED39
:18D9C80000690D690C690B690A24DA3233ED06EC0C38383839303736A9
:18D9E000EE02EC023736EC003736CC0000373630EE0A6F006F016F02DA
:18D9F800C601E703306805690469036902EC0059492509A3062407E312
:18DA1000060C2003A3060DED00EE0A690369026901690024D7303233F4
:18DA2800ED06EE0AEC023838383930EE06EC023736EC003736CE000086
:18DA40003C3C30EE0E6F006F016F02C601E70330680769066905690440
:18DA580069036902690169002529EC02A30CED02E601E20BE701E60090
:18DA7000E20AE7002427EC02E30CED02E601E90BE701E600E90AE70031
:18DA88000C2013EC02A30CED02E601E20BE701E600E20AE7000DEE0E3D
:18DAA000690369026901690024A5303233ED0A3233ED0CEE0EEC0230F7
:18DAB800EE08313131313937363CCE00003C3C30A6053DED02E606A6DB
:18DAD000053DE301ED016900E607A6043DE301ED01A6008900A700E65F
:18DAE80006A6043DE300ED00EC02ED06EC00ED043838383233393736F8
:18DB00003CCE00003C3C30A60D3DED02A60CE6073DE301ED01A60BE637
:18DB1800073DE300ED00A60AE6073DEB00E700A60DE6063DE301ED0187
:18DB30008600A900A700A60CE6063DE300ED00A60BE6063DEB00E700B0
:18DB4800A60DE6053DE300ED00A60CE6053DEB00E700A60DE6043DEBA9
:18DB600000E700303233ED0A3233ED0C31313131EE0A393C3C3C3736C6
:18DB78004F5F30ED04EE02E600EA01EA022620E603272E5A261930EEDE
:18DB900000EC0230EE02ED0238EC0038ED003131313139383820F73083
:18DBA800EE00E600EA01EA02260FE60327075A2608383820E1387EDCE3
:18DBC0005130EE02A60338E6033C3D30ED06EE02A602383CE6033D3014
:18DBD800E305ED05EE02A601383CE6033D30E304ED04EE02A600383C18
:18DBF000E6033D30EB04E704EE02A603383CE6023D30E305ED0586002B
:18DC0800A904A704EE02A602383CE6023D30E304ED04EE02A601383C68
:18DC2000E6023D30EB04E704EE02A603383CE6013D30E304ED04EE0294
:18DC3800A602383CE6013D30EB04E704EE02A60338E6003D30EB02E792
:18DC500002383233ED003233ED0239000000010000000A000000640034
:18DC68000003E800002710000186A0000F42400098968005F5E1003B06
:18DC80009ACA0005F5E10000989680000F4240000186A00000271000B0
:18DC98000003E8000000640000000A000000013C30E306ED063233E984
:18DCB00005E705A904A704393CEC0230E306EE00ED02EC0030E905EEC2
:18DCC80000E70130A904EE00A700383937363C30EC08A302ED08EC0620
:18DCE000E201E707A200A706383233393CEC0230A306EE00ED02EC006A
:18DCF80030E205EE00E70130A204EE00A70038393C3736EC0230EE0096
:18DD1000A302073630EE03A601E60030EE01A2010730A4008AFBA700A2
:18DD2800EE01E2000730A4000631323338393C4353C30001183C073603
:18DD400030E604533206C9000736E704E603533206C900E70332333871
:18DD5800393CEC024353C30001ED020736E601533206C9000736E7016A
:18DD7000E600533206C900E7003839364F0D495A2AFC163239363CC4F7
:18DD88003FCEDD923AE60038333986939FABB7C2CCD6DEE6EDF3F8FC2D
:18DDA000FEFFFFFEFCF8F3EDE6DED6CCC2B7AB9F93867A6D6155493E37
:18DDB800342A221A130D08040201010204080D131A222A343E49556184
:18DDD0006D7A101113141617181A1B1C1D1E1E1F1F1F1F1F1F1F1E1E08
:18DDE8001D1C1B1A181716141311100E0D0B0A080706050403020101D3
:18DE000000000000000101020304050607080A0B0D0E0304040405059C
:18DE180005060607070707070707070707070707070706060505050459
:18DE3000040403030302020201010100000000000000000000000000C0
:18DE480000000101010202020303030304040404040505050505050675
:18DE600006060606060605050505050504040404040303030303020241
:18DE78000202020201010101010101010101010101010202020202036F
:18DE900003030000000000000000000000000000000000000000000074
:18DEA80000000000000000000000070707070707070707070707070700
:18DEC000070707070707070707070707070707070707000102030405BD
:18DED800060708090A0B0C0D0E0F101112131415161718191A1B1C1D8E
:18DEF0001E1F000000000000001004040404050505100000000000009E
:18DF0800000000000000000000083C7C006C7C004ABDE25D3648840E03
:18DF20008AA03716BDE2EABDE2CC4D332627BDE2EABDE2CC4D262230F8
:18DF3800A6008A80BDDF5D4D260AA60084802603BDE2824F7A006C7A08
:18DF5000004A313839860120F3860220EFD615C40226363C7C006C7CEF
:18DF6800004ABDE25D364816C40ECAA1BDE2EABDE2CC4D2618BDE33536
:18DF800030A60084802603BDE28286007A006C7A004A313839860320EA
:18DF9800F38605393C3736CE00003C9615840226667C006C7C004A306C
:18DFB000A6028A80E603BDDF124D264730EE08E700081830ED083808C4
:18DFC8003C30EE040927301830ED046C032721BDE2A7BDE33530EE0852
:18DFE000E700081830ED0838083C30EE0409270F1830ED046C0326DF73
:18DFF800BDE2826C0220B04FBDE28238313131317A006C7A004A3986DD
:18E010000520F096158402266A7C006C7C004A373C30BDE25DA60548E2
:18E0280084AE8AA03616BDE2EABDE2CC4D264030E607BDE2EABDE2CC80
:18E040004D2638E603BDE2EABDE2CC4D2631BDE282C60BD76930BDE29B
:18E058005DE600BDE2EABDE2CC4D2706966926EE8604BDE282313833A5
:18E070007A004A7A006C39860120EF860220EB860320E78605397C00BC
:18E088006C7C004A373C30EC05ED05EE09E60030EE073CBDE013384D55
:18E0A000261730EC09C30001ED09EC07C30001ED07EC0583000126D92D
:18E0B8004F38337A006C7A004A395F4F3736BDDF124D32332607C30048
:18E0D00080810825EF393C3736CE00003C7C006C7C004A30A6028A809F
:18E0E800E603BDDF124D264B30EE08E1002650081830ED0838083C305D
:18E10000EE040927321830ED046C032723BDE2A7BDE33530EE08E1009F
:18E11800262D081830ED0838083C30EE0409270F1830ED046C0326DDCF
:18E13000BDE2826C0220AC4FBDE28238313131317A006C7A004A3986A7
:18E1480004BDE28220ED71E714720410C6B4D740D70171FB03717F03D0
:18E160007210037F004386FEC64ABDE192C608D720D741720815C60C5E
:18E17800D742D716719B177F004D7F004F7F00507F00917F008F7F0060
:18E1900095397C006C7C004A94439743DA43D74386083658251D71FD47
:18E1A800037202409640970171FB409640970171FB037204409640978E
:18E1C00001201871FD409640970171FB409640970171FB03720440961D
:18E1D800409701324A26C371FD4096409701728003717F037A006C7A8E
:18E1F000004A397C006C7C004A4D260F58860658185949184A26F88668
:18E20800122008180505CA0218860F581859491836240971FD40964018
:18E220009701200A71FD03720240964097013671FB409640970101013F
:18E2380071FB037204409640970132324A26CC71FD4096409701720805
:18E2500017010171F7177A006C7A004A393671FD409640970171FB403D
:18E268009640970171FD037202409640970171FB03720440964097010A
:18E2800032393671FD037202409640970171FB409640970171FD4096F4
:18E2980040970171FB037204409640970132393671FD03720240964067
:18E2B000970171FB409640970171FB037204409640970171FD4096408D
:18E2C8009701323971FD409640970171FB4096409701960371FB03728B
:18E2E0000440D640D70184024439373686083658251D71FD0372024001
:18E2F8009640970171FB409640970171FB03720440964097012018714A
:18E31000FD409640970171FB409640970171FB0372044096409701326B
:18E328004A26C371FD4096409701323339363C4F363071FD40964097AE
:18E3400001868071FB40D640D701D603C4025D270616AA00A70017710C
:18E35800FB03720440D640D7014424DF33383239C632D71CC610D71B3B
:18E37000C634D710C606D71EC60AD71139D6B7D1B6270ECE00B23AA659
:18E38800005CC403D7B7164F3986035F39D6B7D1B627FACE00B23AA678
:18E3A000005CC403D7B7164F39D6B0D1AF261286FF5F39D6B0D1AF268F
:18E3B800083FDC8C26F586FF39CE00AB3AA6005CC403D7B0163CCEC2E0
:18E3D0005A3AE6003839369611842027FAD713323937363C966B27037F
:18E3E8003F20F99611842027FAD713961184203F27F9178A10815D270F
:18E40000148A01815F270EC1782506C6A8D76B2004C62AD76B38323349
:18E418003996B690B784033937860136BDE4194D27085A2705BDE3957B
:18E4300020F2C62AD769D6692728BDE4194D26033F20F3BDE395C17F0D
:18E4480026048D22201430E101270CC174270EBDE4194D26E62003309A
:18E460006F00323339C6758670BDE4B920F4BDE39537BDE37D4D27FA01
:18E4780033BDE3E1BDE4A13937363CBDE37D4D2614C1202410BDE41941
:18E490002705BDE39520F2BDE3E1BDE4A13832333917D6AF5CC403D1D8
:18E4A800B0270DD6AFCE00AB3AA7005CC403D7AF3981752606BDE5D91A
:18E4C0007EE57281642606BDE5C17EE572816C2606BDE60B7EE5728109
:18E4D8004C26074FBDE6157EE57281782606BDE5A67EE5728163260388
:18E4F0007EE4FD817026037EE5697EE57296598108246FBDE5794D2760
:18E5080069BDE6D217C47FC02037364F05C3E8CF18EC001833C48018FD
:18E5200027094D27048A102002CA1037364D270D16BDE3E1BDE4204D12
:18E5380026F730E601BDE3E1BDE4204D26F7323116CA10C15D2703331D
:18E5500020208410CEE98D333AE600378B4E16BDE3E1BDE4204D26F776
:18E5680033BDE3E1BDE4204D26F739BDE3D67EE572373C17CE0051D6B9
:18E58000593AA1002712968F840827158670CB60BDE4B971F78F20098E
:18E598007C005972088F4F2002860138333937545454548D0633C40FD1
:18E5B0008D0139C10A2502CB07CB308663BDE4B93937C1642602C064A9
:18E5C800C10A250333200AC6308663BDE4B9332000C10A25264FCE002C
:18E5E0000ABDD9603CC10A25114FCE000ABDD9603CCB308663BDE4B94F
:18E5F8003818CB308663BDE4B93818CB308663BDE4B93917C40F84F058
:18E610003008080808363C37A6002A07BDDD593062700333C4072719EC
:18E628003730C609E200315858CEDC7F3AEC023736EE003CBDDA3238F8
:18E6400038383216C440270616C40F27014A3CC6DA37363CCC000ABD66
:18E65800D9DD18383237E603EA02EA01EA003C36840F2703306A003296
:18E67000385D26DE16C440271116C480270C16C4202704C6FD2002C64A
:18E68800FB3716C40F27134D2B05CE00002003CEFFF01837185A26FA19
:18E6A00084F016C440271116C480260C16C4202704C6FD2002C6FB370E
:18E6B80033C1DA270B36CB308663BDE4B93220F03816C4102703BDDDAE
:18E6D000593937363C17D659C1082409CE00513AA7007C005938323349
:18E6E8003937364F36363636E600271308C125271586633CBDE4B93054
:18E700006F026F033820E9313131313233395F3C30A603A704A602A70D
:18E7180003E70238E60027E708178A2081782752816926037EE8058197
:18E730006426037EE8058173272281632712C12527B7C12B27C9C13AE4
:18E7480024A6C13025A220BF3C30E6056C053AE60A38209D3C30E6051A
:18E76000178B02A7053AEE0AE600270A86633CBDE4B9380820F2387E81
:18E77800E6F03C30E605174C4CA7053AEE0A3C30A6042744E605270438
:18E79000C13027028B80803036C60830EE01A60084F0260D5AA60084A8
:18E7A8000F2606085A26EFC601371730E601C47F10241540C6306D014B
:18E7C0002A02C62036378663BDE4B933324A26F433173130EE00C00855
:18E7D8005037543A3331313CC401260B30EE00E600545454542007389A
:18E7F000E600083CC40F36BDE5B3324A1626E13131387EE6F03C30E6B0
:18E8080005174C4CA7053AEE0A3C30A604271E812B26048640201684B5
:18E820000FE605270EC13026048A80E606C12B26028A4088805F38BD66
:18E83800E615387EE6F03C3736CC0000ED00ED02384FE600C47F274FCA
:18E85000C1302504C13A25113C30EE02E600EA01EA02EA0327323820AE
:18E86800363C36C030375F3737371658584FC3DC8318EC02EE00BDDA03
:18E88000FE313131313C30EE05E302ED023233E901E701A900A70032D2
:18E8980038084C810825AB38393C18C62A3718CE000ABDD96018378CD6
:18E8B000000026F230E60008C12A26F9EE004F33C12A2709CB30E700A3
:18E8C80008A70020F23839004C4E604E214D454D354D284D474E204DC5
:18E8E000714D114F294F284D084D044D014D0800400041004200430013
:18E8F80044004500460047004800494D114D184E144D054D0A4F274DD0
:18E91000754F0D4F0E4F0F4F104F114F124F134F144F154F164F174F00
:18E92800184F194F1A4F1B4F1C4F1D4F1E4F1F4F204F214F224F234FC1
:18E94000244F254F264D714D024D114E05004B4D024F0D4F0E4F0F4FF4
:18E95800104F114F124F134F144F154F164F174F184F194F1A4F1B4FF1
:18E970001C4F1D4F1E4F1F4F204F214F224F234F244F254F264D714E02
:18E98800604D114D220000000A6A0650000003000000080004404142AE
:18E9A00043444546474849000000080000090D0E0F10111213141516B5
:18E9B8001718191A1B1C1D1E1F202122232425260010030000000D0E31
:18E9D0000F101112131415161718191A1B1C1D1E1F20212223242526B3
:18E9E80000000304373CD642CA10D716D74230E6022608D617C4EFD7E8
:18EA0000172006D617CA10D71738333937363CCE00003C3736CC7D00FF
:18EA1800BDD9923838DD9ADE468CEE2C27798CEF5927748CEEC5277424
:18EA30008CEFAA276F8CEDF02773D642C48FD742D716D617C48FD71771
:18EA4800C600D74A0FD6640E01010FD16427F8D60FDC0BDD198307CAFD
:18EA6000C304DEDD0BCC0001DDA04F97A897A99642D617FD0400FD0432
:18EA780002FD0404FD0406FD0408FD040AFD040CFD040EFD0410FD0436
:18EA900012FD0414FD0416CEEDF0FF04182008CEEF592003CEEFAADFC3
:18EAA800467F004A0E3832333937363CCE00003C3736CC9C40BDD99273
:18EAC00032330432463356DDA5DE468CEE2C27448CEDF027318CEF5988
:18EAD800273A8CEEC5272C8CEFAA27300FD642C48FD742D716D617C486
:18EAF0008FD717C601D74AD6640E01010FD16427F8CEEE2C2008CEEF2F
:18EB0800592003CEEFAADF467F004A0E3832333937D696270C363C58A0
:18EB2000CEED823AEC007EEAB4333937363CCE00003C3736CC7D00BDCC
:18EB3800D9923838DD9ACE00003C30EE023CCC7D00BDD9923838DD9EB1
:18EB5000DE468CEEC527538CEDF0273F8CEE2C273F8CEF59273A8CEF45
:18EB6800AA27350FD642C48FD742D716D617C48FD717C600D74AD664C0
:18EB80000E01010FD16427F8D60FDC0BDD198307CAC304DEDD0BCEEEAB
:18EB9800C52008CEEEC52003CEEFAADF460EC601D71838323339373641
:18EBB0003C30E300043736EC00A3020438373618CE00003C3736CC7D7B
:18EBC80000BDD992383805DD9ACE00003C30EE023CCC1F40BDD9923830
:18EBE0003805DD9E38DE468CEEC527538CEDF0273F8CEE2C273F8CEFFA
:18EBF80059273A8CEFAA2735D642C48FD742D716D617C48FD717C60065
:18EC1000D74A0FD6640E01010FD16427F8D60FDC0BDD198307CAC30432
:18EC2800DEDD0BCEEF132008CEEEC52003CEEFAADF460EC601D71838EA
:18EC400032333937363CDE468CEE2C27388CEDF027208CEE61271B8CF3
:18EC5800EEC527168CEF1327118CEF5927078CEFAA27022005CEEE2C91
:18EC70002003CEF057DF46D642C48FD742D7169617848F9717383233B3
:18EC88003937363CDE468CEE2C27168CEF5927078CEFAA2707201DCE2B
:18ECA000EDF02008CEEEC52003CEF057DF46D642C48FD716D74296175B
:18ECB800848F97173832333937363CDE468CF057263ECE00003C373632
:18ECD000CC7D00BDD9923838DD9AD640CA40D740D701C600D74A0FD6F9
:18ECE800640E01010FD16427F8D60FDC0BDD198307CAC304DDDD0BCECD
:18ED0000EEABDF467F004A0E383233393736DC4683EEAB260DCCF0579F
:18ED1800DD46D640C4BFD740D701323339CEED3E583AEC000536CEED2D
:18ED3000723AEE00333CCEED7A3AEC00383903010000000100020100EE
:18ED480001010102020002010202000301030203030303000302030088
:18ED600000000000030302030000000000030103030204B9053805C5C0
:18ED7800066102B90302035403AD0000029E02B602CF02E80302031D1D
:18ED9000033903560375039303B403CE03E8040B04300455047C04A491
:18EDA80004CE04F905260555058505B605EA061F063E06560677068FF4
:18EDC00006B106CA06ED0707072B0746076B078807AE07CB07F3081199
:18EDD800083B085A088508A508D108F3092009430972099709C709ED1A
:18EDF000DC98D39ADD98843FCEA132D603C4011B16583A9642D617C467
:18EE08008FE300DD16D60FDC0BC300F9DD0B960F8420270FDC19C307DF
:18EE2000CADD197A0068DE6308DF633BDCA3D3A5DDA3CEA1F8163A3A0A
:18EE38009642D617C48FE300DD16D60FDC0BC300F9DD0B960F842027F4
:18EE50000FDC19C307CADD197A0068DE6308DF633BDC98D39ADD98CE50
:18EE6800A030163AA600D603C4011B16CEA01A3A9642D617C48FE30040
:18EE8000DD16D60FDC0BC300F9DD0BDCA058492402C853DDA0960F8413
:18EE980020270FDC19C307CADD197A0068DE6308DF633BDC98D39ADD27
:18EEB00098D60384202707CA40D7037EEE0DC4BFD7037EEE0DDC98D38D
:18EEC8009ADD98CEAB4C16C43F3ADC9CD39EDD9C16A600CEAB0CC43F65
:18EEE0003AAB0016C40ECEA01A3A9642D617C48FE300DD16D608DC0BD8
:18EEF800C300F9DD0B960F8420270FDC19C307CADD197A0068DE630835
:18EF1000DF633BDC9CD39EDD9C8440CEA132163ADC98D39ADD9816C425
:18EF28007E3AD603C401583A9642D617C48FE300DD16D608DC0BC30073
:18EF4000F9DD0B960F8420270FDC19C307CADD197A0068DE6308DF636D
:18EF58003BDC98D39ADD98CEAB4C16C43F3ADCA3D3A5DDA3E60084C057
:18EF700049492704C9002004C200200058CEA01A3A9642D617C48FE3E8
:18EF880000DD16D608DC0BC300F9DD0B960F8420270FDC19C307CADD30
:18EFA000197A0068DE6308DF633BDC98D39ADD98CEAB4C16C43F3ADC4E
:18EFB8009CD39EDD9C16A600CEAB4CC43F3AAB0016C40ECEA0183ADCCE
:18EFD000A3D3A5DDA35F4859593A9642D617C48FE300DD16D608DC0B48
:18EFE800C300F9DD0B960F8420270FDC19C307CADD197A0068DE630844
:18F00000DF633B7F006CDC09C307CADD0BC608D708CC0000DD63D76639
:18F01800CB64D76ACEF03DDF46397F00B67F00B7721011393BDE449FE4
:18F030004408357C00483B3B3BDE466E007A0069966B27034A976B7D69
:18F04800006C260BD640C802D740D70171FD03D60FDC0BC307CADD0B8B
:18F060007A0068DE6308DF63D64A26129649D648D749112609DE449FB5
:18F078004408357C00483B3B961116C4402611D61EC410260B16C4807A
:18F09000260916C420262F3BD6123B96120ED6B65CC403D1B7270ED694
:18F0A800B6CE00B23AA7005CC403D7B63BD6B85C26015AD7B8D6B6CEFA
:0DF0C00000B23AA7003B71FB113B3B3B3B0C
:182200000F8E013FC60CD71CC610D71BC624D710C600D71EC60AD71118
:1822180071FB17D642CA06D742D71671F917CC05803716BD02A633BDC9
:1822300002A6CE0539BD029BBD03C1C12025F3CA20C165270BC1702774
:182248002DC17226E57E050ACE055EBD029BBD03C1C13025D5C1382472
:1822600007C030BD04B32009CA20C16126C4BD04AB168D3220BCCE05EC
:182278001FBD029BBD03C1C03027085A26AC720417200371FB17CE0503
:182290002D8D08BD02C58D0E7E0232E6002706BD03E30820F639373629
:1822A8003C3786103D168D07338D0438323339C40FCB30C13A2602CBD8
:1822C00007BD03E339301883003218353C3C3C36BD037A813A26F9BD1E
:1822D80003B530E700E702BD03B530E703EB02E702BD03B530E704EB56
:1822F00002E702BD03B517AB02A702C101274A5D26CE30A60027196F00
:1823080001BD03B51730E601EE053AA70030AB02A7026C016A0026E9D9
:18232000BD03B530EB022619EC0537364FE601E3053736EC033736BDD2
:1823380003F0383838C62B2002C62DBD03E37E02D0BD03B5C1FF26F1AD
:18235000CE0362BD029B323838383018C300321835390A0D4F4B008119
:182368003A2504845F8007803058585858361B16323937BD03C1C11B1A
:18238000272AC110271CC1132718C1302514C13B2517C141250CC14730
:18239800250FC1612504C16725073338CE02D03C371733393338CE031D
:1823B000563C3720F4388DC28DAD168DBD8DA83C39BD03DABD042A4D9B
:1823C80027F7398D0DBD042A4D27F836378D0C3332399611849027022D
:1823E000D6123996118420BD042A4D27F6D7133930EC02830200253108
:1823F800EC0283200025037E0443EC063736EC043736EC023736308D7B
:1824100019EE04E60038E700083C30EC04C30001ED04A30226E9383867
:18242800383937D640CA02D740D70171FD03010101D640C4FDD740D7EA
:1824400001333930EC063736EC043736EC02373630EE04E6008D1338F0
:18245800083C30EC04C30001ED04A30226EB3838383930EE02377202F1
:1824700017C6AAF7555553F72AAA86A0B7555533E70071FD1717BD0410
:182488002AA8002A11A600842026F317A80027068D0686FF20014F391F
:1824A000C6F0720217E70071FD1739CE5555C6104F20104F54465446EE
:1824B8008B2071FB17375F18C630323736720217C6AAF7555553F72A8B
:1824D000AA8680B7555553F7555553F72AAA324D270372041733E70081
:1824E80086644A26FD71FD17BD042AA6002B0E842027F5A6002B068D12
:182500009F867720014F71FB1739CE88003CCE90003CCE08003C71FB51
:1825180017BD03F07E080042616E6B3F2028302F31290A0D0053656E65
:18253000642066696C650A0D000A0D52656164792E0A0D0A0D45202D5E
:182548002045726173650A0D50202D2050726F6772616D0A0D00302D4B
:1825600037202D20536563746F72202831366B42290A0D412020202DE5
:1825780020436869700A0D00CE22003CCE25803CCE02003CBD23F07E5B
:0A25900002007204173971FB1739BD
:00000001FF
